:04000000B601932989
:100008000800B616B61EB612B6190E28B615472041
:10001800031835280830A3005B20A20DA30B102875
:10002800B61E402065206120B61A35203A202208E5
:1000380003108E29B616B61EB61236192828FE39B0
:10004800B700361503108E29361A3028A600361642
:1000580047200318352826084E2003183528B61ED1
:100068008E294020652036113612B6113A088400D0
:1000780038088417800446283A088400380980051F
:100088008417800508003A20652040206120370841
:10009800B6190138A2000830A300A20D03183A20AF
:1000A800031C402065206120A30B51283A206520BD
:1000B8003A08840038080005FF3E3B0884003909E7
:1000C80043283B08840039083D282C08A0002D0847
:1000D800A1000130A20064009520031C8228A20B15
:1000E8006F28FF30A007031CA107031C8E29FA30D4
:1000F800A2006F286400952003187E28E720A80135
:100108000830A300E82095200318A80AAB1EA80110
:10011800A20CA30B8628AB1AA213E820031422080A
:1001280008003A08840038088417800484130005FE
:100138002B1B3806FF3E0800A400290803140319E6
:100148008E298921031C0800A0002518831724087C
:100158008400200880008313A40AA903A1280408A6
:10016800A6003A088400F030B7050830A70003104D
:100178000318B70ACD20A60CA70BBC280000AB1AA1
:10018800370CCD2091210314CD202F08A3002E0871
:100198002D298413AB1FDC28000838042B1F3806D0
:1001A8008000841700083804031C38068000E828FB
:1001B80000083804031C38062B1B380680008417F7
:1001C80038098005E82837172B081F39003EA10099
:1001D8002A080E3E0318A10A371F3A293713A00030
:1001E800023054213A29B71329080319B7170530E3
:1001F800A8002730A30010300D210330A300E830F9
:100208000D21A30164300D21A3010A300D2124081A
:100218001429A2002508A1002408A0006D212008A7
:10022800A000A8030319B713290803191E292802D7
:10023800031808002008031DB713B71B0800303E39
:10024800892983178001840AFF3E031D26298E29E8
:10025800A301A200FF30A207031CA307031C8E29D9
:100268000330A100E7303A212E29A101FC3EA0006D
:10027800A109031C4529FF300000A00703184029E5
:10028800A0076400A10F3F2908000310A00DA10DCD
:10029800FF3E0318492920088E290310A10CA00C41
:1002A800FF3E0318512920088E29A301A20001301E
:1002B8005D29A80023082102031D642922082002C1
:1002C800043003180130031902302805031DFF30DC
:1002D8008E291030A600A501A401210DA40DA50D9D
:1002E8002208A4022308031C230FA502031883294C
:1002F8002208A40723080318230FA5070310A00D3D
:10030800A10DA60B712920088E29840031088A00C6
:10031800300882008313031383126400080020301E
:10032800840060308A012621A030840050308A0180
:1003380026211030840060308A0125219030840005
:1003480060308A012521831607309F0099018312A6
:100358009801831602309800B701B801861006117B
:1003680088010710871007118312071186100130C2
:100378008A012C21861464308A012C218A110A12E0
:10038800D82B071083162608831288008A110A12B0
:10039800D2290714831628088312880087100000C2
:1003A80087140710080083164630A80083128A01B4
:1003B800CD218316A60183128A01C5218316103028
:1003C800A60083128A01C52183164C30A800831227
:1003D8008A01CD2183164230A80083128A01CD21DB
:1003E8008316A6010130AB008312640081308316A6
:1003F8002B028A110A12831203181F2A831601304E
:10040800AE0083126400213083162E028A110A126C
:1004180083120318182A8A01C5218316AE0A8A1185
:100428000A128312031D062A8316AB0A8A110A12BE
:100438008312031DF92983164630A80083128A0106
:10044800CD218316A60183128A01C5218316103097
:10045800A60083128A01C52183164C30A800831296
:100468008A01CD21080083164630A80083128A012C
:10047800CD218316A60183128A01C5218316103067
:10048800A60083128A01C52183164C30A800831266
:100498008A01CD21080083164630A80083128A01FC
:1004A800CD218316A60183128A01C5218316A601D0
:1004B80083128A01C52183164C30A80083128A0151
:1004C800CD2183164230A80083128A01CD218316DC
:1004D8000130AB0083126400113083162B028A119D
:1004E8000A1283120318992A83160130AE00831268
:1004F8006400213083162E028A110A12831203180F
:10050800922A83162030A60083128A01C5218316F9
:10051800AE0A8A110A128312031D7C2A8316AB0ABB
:100528008A110A128312031D6F2A83164630A80007
:1005380083128A01CD218316A60183128A01C5215F
:100548008316A6014C30A80083128A01CD21080029
:1005580083164030A80083128A01CD218316AB018F
:1005680083126400083083162B028A110A12831240
:100578000318E62A83162B08073C8A110A128312ED
:10058800031CDD2A8A110A12CF228316A6008312C1
:100598008A110A12DD2A02308A0083162B08831278
:1005A80082073034873407341F3452347F34203480
:1005B80000348A01C5218316AB0A8A110A128312F4
:1005C800031DB52A83164430A80083128A01CD2161
:1005D8008316AB0183126400063083162B028A113E
:1005E8000A12831203181E2B83162B08053C8A1146
:1005F8000A128312031C152B8A110A120923831667
:10060800A60083128A110A12152B03308A0083165A
:100618002B0883128207003400347F3400341034EE
:100628007F348A01C5218316AB0A8A110A12831204
:10063800031DEF2A83165A30A80083128A01CD21A0
:100648008316A60183128A01C52183165B30A80090
:1006580083128A01CD2183160130A60083128A01F4
:10066800C52183165830A80083128A01CD2183162C
:100678001630A60083128A01C5218A01D7218A0172
:100688004F2283164630A80083128A01CD21831693
:10069800A60183128A01C5218316A60183128A0145
:1006A800C52183164C30A80083128A01CD218316F8
:1006B8004230A60083128A01C5218316A60183123F
:1006C8008A01C52183165D30A80083128A01CD21D5
:1006D80083160430A60083128A01C521831686304A
:1006E800A60083128A01C52183165930A8008312F7
:1006F8008A01CD2183161430A60083128A01C521F0
:1007080083164C30A80083128A01CD210800831675
:100718002B083C3E840000088312B200FF30A20080
:10072800A20A22080F3C8A110A12031CBE2B8A1146
:100738000A12AA2332028A110A12031D942B2208D4
:100748008316B30083128A110A12BE2B03308A0063
:100758002208820730343134323433343434353477
:100768003634373438343934613462346334643479
:1007780065346634080083164630A80083128A015F
:10078800CD2175088316A60083128A01C521760833
:100798008316A60083128A01C52183162908A8009A
:1007A80083128A01CD2108008A01AC22C530F500E8
:1007B800F60183164C30A90083128A01BF238316E1
:1007C8004230A80083128A01CD218316AB0183121F
:1007D8006400163083162B028A110A12831203183A
:1007E8002B2C83162B08153C8A110A128312031C22
:1007F800222C8A110A1206248316A60083128A1153
:100808000A12222C04308A0083162B0883128207CE
:10081800503449344334203443346F346E347434A0
:1008280072346F346C346C3465346434203453342B
:100838004534443431343334333430348A01C521B7
:100848008316AB0A8A110A128312031DEC2BE330BC
:10085800F500F60183164C30A90083128A01BF23E4
:1008680083164230A80083128A01CD218316AB017A
:10087800831264001B3083162B028A110A1283121A
:100888000318812C83162B081A3C8A110A1283122A
:10089800031C782C8A110A1257248316A600831287
:1008A8008A110A12782C04308A0083162B088312C6
:1008B80082075534733469346E34673420345034C5
:1008C8006934633442346134733469346334503482
:1008D80072346F3420345634653472342E342034F4
:1008E80032342E34333432348A01C5218316AB0AAC
:1008F8008A110A128312031D3D2C0530F5000130C0
:10090800F60083164C30A90083128A01BF23831690
:100918004230A80083128A01CD218316AB018312CD
:100928006400153083162B028A110A1283120318E9
:10093800D22C83162B08143C8A110A128312031C2A
:10094800C92C8A110A12AE248316A60083128A11B2
:100958000A12C92C04308A0083162B0883128207D6
:10096800523461346E346A34693474342034443413
:1009780069346F346C3420342D34203443344F348C
:100988004D3450345334793473348A01C521831675
:10099800AB0A8A110A128312031D942C2430F50025
:1009A8000130F60083164C30A90083128A01BF2358
:1009B80083164230A80083128A01CD218316AB0129
:1009C80083126400173083162B028A110A128312CD
:1009D8000318252D83162B08163C8A110A12831238
:1009E800031C1C2D8A110A12FF248316A6008312E9
:1009F8008A110A121C2D05308A0083162B088312CF
:100A0800820768347434743470343A342F342F3491
:100A18007734773477342E3463346F346D347034EC
:100A280073347934733431342E3463346F346D3421
:100A38008A01C5218316AB0A8A110A128312031D83
:100A4800E52CF5011030F60083164F30A90083120B
:100A58008A01BF2383164230A80083128A01CD2160
:100A680083168030A600AB018312640080308316A1
:100A78002B028A110A12831203184B2D8A01C521F1
:100A88008316AB0A8A110A128312031D392D1F30EF
:100A9800F5001030F60083164F30A90083128A0142
:100AA800BF2383164230A80083128A01CD21831602
:100AB8000130A600AB0183126400803083162B023C
:100AC8008A110A1283120318722D8A01C52183160E
:100AD800AB0A8A110A128312031D602DF50110302A
:100AE800F60083164C30A90083128A01BF238316AF
:100AF8004230A80083128A01CD218316FF30A60058
:100B0800AB0183126400203083162B028A110A126B
:100B180083120318982D8A01C5218316AB0A8A11FE
:100B28000A128312031D862DE030F5001F30F600EF
:100B380083164C30A90083128A01BF2383164230E2
:100B4800A80083128A01CD218316FF30A600AB01CD
:100B580083126400203083162B028A110A12831232
:100B68000318BF2D8A01C5218316AB0A8A110A1200
:100B78008312031DAD2D8316AE01AB01AF018312A5
:100B88002030FF0083160A30AA008312F501F6010F
:100B9800FD01FE018316A001A1017830AC00AD0172
:100BA80083120730BA008030B8002030AA00AB01A9
:100BB8008A017E202A3C8A110A12031DDC2D093085
:100BC800A9007E30B000B101A5016B308A01A020D8
:100BD8008316AB0183126400093083162B028A1135
:100BE8000A1283120318372E83162B086B3E8400D3
:100BF80000088312B200FF30A200A20A22080F3CAC
:100C08008A110A12031C2B2E8A110A121726320285
:100C18008A110A12031D012E22088316B3008312BB
:100C28008A110A122B2E06308A00220882073034D5
:100C38003134323433343434353436343734383468
:100C48003934613462346334643465346634831609
:100C58002B086B3E840033088000AB0A8A110A1205
:100C68008312031DEF2D7208A000A10104308A0130
:100C78004C21B2002108B300730832048316AA007D
:100C880083126C08A000A10104308A014C21B20033
:100C98002108B3006D083204FF006E08A000A1010E
:100CA80004308A014C21B2002108B3006F083204D5
:100CB800F6007008A000A10104308A014C21B2009E
:100CC8002108B30071083204F5007508F3007608AE
:100CD800F4006B088316AE0064002E08003C8A15E9
:100CE8000A12831203190D28640083162E08013C8A
:100CF8008A110A1283120319342F640083162E08EE
:100D0800043C8A110A1283120319952E6400831673
:100D18002E08053C8A110A1283120319A32E8A0190
:100D2800D52D8316E830AC00AD018312FD01FE011C
:100D38008316A001A10183128A150A1222288A01AA
:100D48004F227F038316AC002A03AD008312FD01F6
:100D5800FE018316A001A10183128A01372283169E
:100D68004230A80083128A01CD21FD01FE017D08D1
:100D7800A0007E08A10083162C0883128A0159213D
:100D88008A110A12031D082F8316A001A1018312DC
:100D9800831620088312A000831621088312A1005D
:100DA80083162D0883128A0159218A110A12031DFC
:100DB800012F0730BA001030B8000730BB000830E8
:100DC800B900A0308A01202074088A012020730805
:100DD8008A0120208A0105208316A60083128A0131
:100DE800C521F30A0319F40A8316A00A0319A10AF4
:100DF8008A110A128312031DCC2EFD0A0319FE0A5A
:100E08008A110A12031DBB2E0730BA004030B80001
:100E18002030AA00AB01AE01AF0144308A01B420F2
:100E280069308A01B42073308A01B42070308A0195
:100E3800B4206C308A01B42061308A01B420793042
:100E48008A01B42065308A01B42064308A01B42054
:100E58000A308A01B4200D308A01B4208A01D52DC8
:100E68000730BA008030B8002030AA00AB018830C3
:100E7800AC001330AD008A0169208A150A12031CE0
:100E8800B1285D3C8A110A12031D3F2F7F08A90073
:100E98006930B000B101A5013C308A01A0208A1553
:100EA8000A12031CB1288316AB018312FF307F0797
:100EB800B400FF300318013EB50083162B088312D7
:100EC800A000A1013508A30034088A015A218A111B
:100ED8000A12031DAE2F83162B083C3E840000081F
:100EE8008312B200FF30A200A20A22080F3C8A1126
:100EF8000A12031CA22F8A110A128E2732028A11A3
:100F08000A12031D782F22088316B30083128A1150
:100F18000A12A22F07308A0022088207303431349F
:100F2800323433343434353436343734383439346D
:100F380061346234633464346534663483162B0850
:100F48003C3E840033088000AB0A8A110A128312DF
:100F5800031D5A2F8316AB018312FF307F07B4009D
:100F6800FF300318013EB50083162B088312A0003A
:100F7800A1013508A30034088A015A218A150A12EA
:100F8800031D0B2883162B083C3E8400000883129F
:100F9800B2003208A000A10104308A014C21B2003D
:100FA8002108B300013083162B078312B400B50162
:100FB800B50D34083C3E84000008B40034083204FF
:100FC8008316A60007308312BA001030B800073025
:100FD800BB000830B900A0308A01202074088A01BB
:100FE800202073088A0120208316260883128A018C
:100FF8001E200A308A012C21F30A0319F40A023050
:101008008316AB078A110A128312031CB12F8A01B7
:10101800342F8A014F228316F830AC00AD018312B9
:10102800FD01FE018316A001A10183128A01372266
:1010380083164230A80083128A01CD210730BA00F6
:101048008030B8002030AA00AB01D030AC000730A7
:10105800AD008A0169208A110A12031CD52D5D3C56
:101068008A150A12031D2D287F08A9006930B000CF
:10107800B101A5013C308A01A0208A110A12031C83
:10108800D52D8316AB018312FF307F07B400FF30E4
:101098000318013EB50083162B088312A000A10196
:1010A8003508A30034088A015A218A150A12031D3B
:1010B8006B288A018B2383162B083C3E8400330857
:1010C8008000AB0A8A150A128312031D482883166A
:1010D800AB018312FF307F07B400FF300318013ED5
:1010E800B50083162B088312A000A1013508A300C0
:1010F80034088A015A218A150A12031DAE2883165C
:101108002B083C3E840000088312B2003208A0007D
:10111800A10104308A014C21B2002108B30001303A
:1011280083162B078312B400B501B50D34083C3E75
:1011380084000008B400340832048316A600831221
:101148008A01C52102308316AB078A150A12831259
:10115800031C6E288A150A1222280730BA0040306C
:10116800B8002030AA00AB01AE01AF016C308A0193
:10117800B42061308A01B42073308A01B4207430FD
:101188008A01B42020308A01B42062308A01B42058
:1011980079308A01B42074308A01B42065308A011C
:1011A800B42020308A01B42061308A01B420743020
:1011B8008A01B4203A308A01B420A9017308A40036
:1011C8007408A500B330B000B1018A01F7200A30D5
:1011D8008A01B4200D308A01B4208A01D52D63001C
:0611E8008A150A12F3282B
:02400E00753DFE
:00000001FF
